:10000000830100308A0004288301412A831294006E
:10001000951B112815088A001408940A0319950ADB
:1000200082008313151883171408940A84000008AB
:100030000800483465346C346C346F343A342034FE
:0200400000348A
:1003340083128F0006168312282A831205110130B6
:100344008312BD2983128F000612803E8312282A4D
:10035400831206120130831228220230BD2983122F
:100364008C0004308D00FA308312BD218D0BB52929
:100374008C0BB32908008312900004309100533091
:100384009200920BC329910BC129900BBF2908003D
:100394008312061221308F008F0BCE29283083124E
:1003A40028220C30282206302822792BE229100832
:1003B40095000F088F0A0319900A0620831203235D
:1003C4008312100895000F0806200038031908004E
:1003D400D9298312AA210616F7290D0895000C08BD
:1003E4008C0A03198D0A062028220D0895000C0892
:0C03F4000620003803190800EF298312CE
:1004000006160B2A0D0895000C088C0A03198D0A94
:100410000620831228220D0895000C0806200038BB
:1004200003190800022A40308312A4210616202A4C
:100430000D0895000C088C0A03198D0A0620282245
:100440000D0895000C080620003803190800182A2A
:1004500083129000100E0F3993000608F039130430
:1004600086008616861210080F3993000608F039A8
:1004700013048600861686120D309100910B3E2AD9
:10048000080083128D018E010830831685008601D5
:1004900083129F21CA2119308F0000309000D8218B
:1004A0008D018E017E228D0A03198E0A00300E0204
:1004B000023003190D02031C522ABF228D018E0146
:1004C0007E228C0003238D0A03198E0A00300E024F
:1004D000023003190D02031C602AAA218D018E012E
:1004E0007E228C009A218D0A03198E0A00300E029A
:1004F000023003190D02031C702A042883128F0195
:10050000851D802A29309000900B842A851D0F14A8
:1005100021309000900B8A2A851D8F142130900085
:10052000900B902A851D0F1521309000900B962A74
:10053000851D8F1521309000900B9C2A851D0F166C
:1005400021309000900BA22A851D8F16213090003B
:10055000900BA82A851D0F1721309000900BAE2A12
:10056000851D8F1721309000900BB42A2130900008
:10057000900BB82A0F08831203230F080800831278
:10058000AA2100309A2103309A2105309A210530A2
:100590009A2105309A2100309A2103309A210030A7
:1005A0009A2103309A2105309A2105309A21003092
:1005B0009A2103309A2105309A2105309A2103307F
:1005C0009A214030A42120309A2106309A2105300A
:1005D0009A2100309A2103309A2105309A21023065
:1005E0009A2120309A2106309A2100309A21043035
:1005F0009A2101309A2107309A2104309A21013042
:100600009A2107309A29831291009109051521300A
:100610009200920B092B110C031C102B0515112BAA
:10062000051103108312910C21309200920B162BAE
:10063000110C031C1D2B05151E2B05110310831215
:10064000910C21309200920B232B110C031C2A2BAE
:1006500005152B2B051103108312910C21309200EC
:10066000920B302B110C031C372B0515382B051161
:1006700003108312910C21309200920B3D2B110C30
:10068000031C442B0515452B051103108312910CF7
:1006900021309200920B4A2B110C031C512B051593
:1006A000522B051103108312910C21309200920BF2
:1006B000572B110C031C5E2B05155F2B0511031026
:1006C0008312910C21309200920B642B110C031CAD
:1006D0006B2B05156C2B051103108312910C213027
:1006E0009200920B712B051121309200920B762B08
:1006F00008008312061240308312282206160030AA
:1007000028220030282200302822043028220230FB
:1007100028221F30282202302822043028220030CC
:1007200028220030282200302822043028220830D5
:1007300028221F30282208302822043028220430A2
:1007400028220E30282215302822043028220C308E
:100750002822183028220030282200302822003099
:10076000282200302822003028220E302822113082
:10077000282211302822113028220E302822003061
:10078000282200302822003028220E302822113062
:10079000282215302822113028220E30282200303D
:1007A0002822003028220030282200302822003061
:1007B00028221F302822003028220030282204302E
:1007C000282204302822043028220430282206302F
:1007D000282203302822003028220030282204302A
:1007E00028220430282204302822043028220C3009
:1007F0002822183028220030282200302822AA2956
:02400E00F93F78
:00000001FF
